:1000000000308B0010308500003086008316C5302C
:100010008100043085000030860000309A00831291
:10002000103084008001840A841E1228041E1228C5
:100030000D22213075239D0024307523A00022302D
:100040007523A700A200233075239B009B18AB14D7
:100050009B181B150430A4002B120510DD21B020C5
:10006000A6206C20EF2032222F284420051D3528A1
:100070003E200310051D08000314080004309900F9
:100080004420990B402808000B1D49280B11A90A90
:100090004C280000000000001A185D288611010895
:1000A0009C001C0C7F39031959281E02031C0611E1
:1000B00008009E08031D06150800061101089C0093
:1000C0001C0C7F39031968281E02031C86110800C6
:1000D0009E08031D8615080014089000150891005D
:1000E0001608920017089300940195019601970154
:1000F000143084007E20872091200800083098006A
:10010000051980283520800D980B80280800840A66
:10011000051988283520800D05198C283520800D7B
:100120000800840A04309800051994283520800CB2
:10013000840A051999283520800C98030319A228F0
:1001400084039428800E8403800E0800093005196A
:100150000D3E99000519A6284420990BAA280800ED
:10016000AB1CEC28AB19BB28A1080319BE28DE2064
:100170000514AB15E2280000000000000518CD288A
:1001800029082C02031DE72805142908AB1DCA28DD
:100190001B18203E203EAC00080029082C02031D3D
:1001A000E42805101E080319AB11AB1DDE28AC00B6
:1001B0001B18AC0D2C082902AC0008002908AC0063
:1001C000AC03080000000000000000000000000078
:1001D00000000000000008009B18051044281008CB
:1001E0001402031D0F2911081502031D0F291208FF
:1001F0001602031D0F2913081702031D0F291B1FC9
:100200000529100820020319092910081D02031DE1
:100210000F2944201208130203199F2910290800EE
:100220002B1697089703970303193A299703031985
:10023000061397030319861397030319402997039D
:1002400003198921970303197421970397039703CF
:1002500003194529970303190617970303198617EE
:10026000970303193D299703031994219703031951
:100270007F21B6291208073C6B291208F83E6B292A
:100280001208073C03185B296B2908309602031CEF
:100290006B2903190F299603960396030319061772
:1002A0009603031986179603960303199421960360
:1002B00003197F21B629013E03197421013E031958
:1002C0008921013E013E03198613013E03190613DD
:1002D000013E013EB629130803391A060319B6294F
:1002E000130803399A00B6299B1E7D29A8002230E5
:1002F0007523A700A20028080800851008009B1E8F
:100300008729A8000130A700A2002808080085144A
:1003100008001B1D92299B1C9029AB142B1108006F
:100320002B110800051008001B1D9D299B1C9B29F3
:10033000AB102B1108002B1508000514080012083B
:10034000013A031DB3291B18A929FF30A30004306B
:10035000A4001B1843221B18B6291B149A0901304C
:100360009A052822B6291B1CB6291B104420DD2122
:100370001208013A0319DA291208AA002B19CD290B
:100380000310AA0D9B1FD12991080319D129111C13
:10039000AA0A9118D129AA0AD1292B1ED1293030B5
:1003A000AA072A087523A1002A081F0203190800BA
:1003B00021220800A1019E0108001B1AFF291A181A
:1003C000F029061286169E08031986129B1D8616B2
:1003D0002B1A08009118EE290613080006170800CA
:1003E000861206169E08031906129B1D06162B1A66
:1003F00008009118FD2986130800861708001A18AE
:10040000072A061291188616911C86120800861279
:1004100091180616911C06120800203075239F00C3
:100420009F1A2B151B191A2A0F309F052B11031029
:100430009F0D1F0875239E00A100253075239A008B
:100440000800203089002A089F00880068230800DF
:10045000253089001A0888006823831688182E2AF8
:10046000831208002B1221081E0203190800A20B98
:10047000080021081E02031C3F2A9E03402A9E0AF0
:100480002708A2000800A30B0800472A0800FF3035
:10049000A300A40B0800792A0B30A50B502A0800F2
:1004A000861606167B23861206127B234D2A0230FF
:1004B000A5002F304D2A66221208013A03195B2A43
:1004C00066221208013A031D602A0800A6206C204B
:1004D00010081402031D662A11081502031D662A5E
:1004E00012081602031D662A13081702031D662A46
:1004F00008000A30A5004C220230A5004C225B22E5
:100500008323A8030319A12AA8030319AB2AA8036C
:100510000319B62AA8030319F72AA80303190D2BF8
:10052000A8030319442BA80303194E2BA80303198E
:100530001F2BA8030319322B10080319602B572215
:100540007F2A0230A5004C225B222130890010084E
:10055000880068237C2A0330A5004C225B222230CD
:10056000890083232808880068237C2A0430A5009A
:100570004C225B228323280889000310890D100870
:100580000319DC2A10302802031CC82A5722B92A72
:100590002808A500A50A4C225B221008832303101B
:1005A000A80DA81FD52A5722CC2A2808880068231E
:1005B0000230A5004C22B92A0630A5007523A800F8
:1005C000A50325037523A8020310280C8807250816
:1005D0008900682383168818EB2A8312A50A1E3027
:1005E000250203187C2AA50AA50A2508DE2A05305B
:1005F000A5004C225B22832304302802031C022B1B
:100600005722FA2A23307523E7308805A8032818D3
:100610008815A818081668237C2A0630A5004C22E5
:100620005B22832303302802031C182B5722102B34
:10063000233075238812281C881668237C2A0930E9
:10064000A5004C225B22832305302802031C2A2BA1
:100650005722222B23307523F83088052808880478
:1006600068237C2A0A30A5004C225B2283230330B6
:100670002802031C3D2B5722352B2330752388136A
:10068000281C881768237C2A0730A5004C225B228F
:10069000243089001008880068237C2A0830A500CF
:1006A0004C225B22832303302802031C592B572240
:1006B000512B233075230813281C081768237C2A24
:1006C000FF30A3000430A4000B30A5004C221228F8
:1006D00083168B1308128811081555308900AA302B
:1006E00089008814081183120800890083160814F1
:1006F0008312080808000B11A6000B1D7D2B0B119F
:10070000A60B7D2B0800A801901F892BA80A101F9B
:10071000A80A901E8F2B0330A807101EA807901D53
:10072000952B0930A807101DA807901C08001B3046
:08073000A807101CA80708002F
:02400E00FB3F76
:104200000000000000000000140015001600180057
:104210001A001C001E0020002200250028002B0090
:104220002E00320036003A003E00430048004E00A7
:1042300054005A00600067006E0075007C000000AA
:1042400000002A0001002000A9000000000000007A
:10425000000000000000000000000000000000005E
:104260000000000008000A000C000E001000120000
:10427000150018001B001E002100250029002D003C
:00000001FF
